:020000040000FA
:0600000029EF22F01200BE
:020006001200E6
:0600080025EF0AF01200D2
:060018001AEF01F01200D6
:02001E000100DF
:0C0020008444000000010000D200000039
:04002C00948E949C7E
:10003000200EAF6EAC8AAC84AC9CAB8EAB889E9825
:100040009D8AF28EF28C1200D9CFE6FFE1CFD9FF64
:10005000E65200016251601902E16351611901E148
:10006000F8D760C0E9FF61C0EAFF602B000E612392
:10007000EFCF00F0016A00BE01680050DF6E280E6D
:10008000605D010E615904E3000E606F010E616F47
:10009000DF5000D0E552E552E7CFD9FF1200D9CFAB
:1000A000E6FFE1CFD9FF020EE126DE6ADD6AAC5041
:1000B000020B01E0010E006E016A0050011010E118
:1000C000DF2A010E01E3DB2AD9CFE9FFDACFEAFF0D
:1000D000E80ED880EE54030EED5401E20ED0E7D7BF
:1000E000FE0EDB50AD6E9E50100B01E0010E006E57
:1000F000016A0050011001E1F6D7020EE15C02E254
:10010000E16AE552E16EE552E7CFD9FF1200D9CF9F
:10011000E6FFE1CFD9FF030EE126FD0EDBCFDEFFC8
:10012000DBCFDDFF91DFE76E020EE7CFDBFFDBCF3A
:1001300000F0016A00BE0168FC0EDBCF02F0036A2A
:1001400002BE03680250001802E10350011812E0D9
:10015000020EDBCF00F0016A00BE0168FD0EDBCFAE
:10016000E9FFDB2AFE0EDBCFEAFF01E3DB2A00C05A
:10017000EFFFD8D7FD0EDBCFE9FFFE0EDBCFEAFFA6
:10018000EF6ADECF00F0DDCF01F000C0F3FF01C069
:10019000F4FF030EE15C03E200D0E16AE552E16E98
:1001A000E552E7CFD9FF1200D9CFE6FFE1CFD9FF63
:1001B000020EE126DE6ADD6AFD0EDBCFE9FFFE0EF0
:1001C000DBCFEAFFEFCF00F0016A00BE016800500C
:1001D000011019E0FD0EDBCFE9FFFE0EDBCFEAFFD9
:1001E000EFCF00F0016A00BE01680050E66E57DFF5
:1001F000E552DF2A010E01E3DB2AFD0EDB2AFE0EAB
:1002000001E3DB2AD9D7010EF36EF46A020EE15C3A
:1002100003E200D0E16AE552E16EE552E7CFD9FF93
:1002200012000D0EE66E3BDFE5520A0EE66E37DF7A
:10023000E5521200DACFE4FFE2CFDAFFE9CFE4FFC4
:10024000EACFE4FFE652D9CFE6FFE1CFD9FFE6528D
:100250009E50200B01E0010E306E316A305031109B
:100260001BE0AE50DF6EDFCF30F0316A30BE316858
:10027000000162C0E9FF63C0EAFF622B000E632346
:1002800030C0EFFF280E625D010E635904E3000EDB
:10029000626F010E636F9E9AE552E552E7CFD9FF78
:1002A000E552E5CFEAFFE5CFE9FFE5CFDAFF110040
:1002B000D9CFE6FFE1CFD9FFFE0EDB50006E016A19
:1002C000013404E200500008000E015403E2FE0E67
:1002D000DB06F2D7E552E7CFD9FF1200D9CFE6FF10
:1002E000E1CFD9FFFE0EDB50E66EECEC21F0E552DB
:1002F000E552E7CFD9FF1200D9CFE6FFE1CFD9FF12
:10030000030EE126FE0EDB50006E016A013404E2AA
:1003100000505F08000E015401E2A3D0FD0EDB5037
:10032000006E016A013404E200503F08000E0154DF
:1003300001E297D0FD0EDB50026E036A080E256EB7
:10034000266A02C020F003C021F0F5EC1BF020C0AB
:1003500002F021C003F0600E0302F3CF03F00202AB
:10036000F3CF02F0F4500326FE0EDB50000102240E
:10037000006E000E0320016E00C0DEFF01C0DDFF35
:10038000FD0EDB50026E036AFD0EDB50046E056A43
:10039000080E256E266A04C020F005C021F0F5EC99
:1003A0001BF020C004F021C005F0030ED8900436E5
:1003B0000536E806FBE10450025C006E0550035868
:1003C000016E020E00C0DBFFFC0EDB50006E016A06
:1003D0000050011014E1020EDB5037EC22F0F3CF95
:1003E00000F0F4CF01F0001E011EDECFE9FFDDCFEB
:1003F000EAFF830EE926000EEA220050EF16FC0EFB
:10040000DB50006E016A010E001801E1015010E19D
:10041000020EDB5037EC22F0F3CF00F0DECFE9FF25
:10042000DDCFEAFF830EE926000EEA220050EF122C
:10043000FC0EDB50006E016A020E001801E1015053
:1004400010E1020EDB5037EC22F0F3CF00F0DECFEC
:10045000E9FFDDCFEAFF830EE926000EEA22005015
:10046000EF1A030EE15C02E2E16AE552E16EE55249
:10047000E7CFD9FF1200D9CFE6FFE1CFD9FF0A0EAF
:10048000E126FB0EDB50026E036AFD0EDB50046EAC
:10049000056A0450025C006E05500358016E020E9E
:1004A00000C0DBFF030E01C0DBFFFC0EDB50026E61
:1004B000036AFE0EDB50046E056A0450025C006E97
:1004C00005500358016E00C0DEFF01C0DDFF020EC3
:1004D000DBCF00F0030EDBCF01F00001800E011432
:1004E00015E020682168020EDBCF25F0030EDBCF7C
:1004F00026F01BEC1CF0020E1EC0DBFF030E1FC01B
:10050000DBFF060EDB68070EDB6807D0010EF36E1B
:10051000060EF3CFDBFF070EDB6ADECF00F0DDCF88
:1005200001F00001800E011411E020682168DECF87
:1005300025F0DDCF26F01BEC1CF01EC0DEFF1FC037
:10054000DDFF040EDB68050EDB6807D0010EF36EDD
:10055000040EF3CFDBFF050EDB6AD9CFE9FFDACF5C
:10056000EAFF010ED890EE36ED36E806FBE1D950F1
:10057000020FE96EDACFEAFF010ED890EE36ED36C3
:10058000E806FBE1FA0EDB50E66EFD0EDB50E66E90
:10059000FE0EDB50E66EB0DEE552E552E552DECFF0
:1005A00000F0DDCF01F0020EDBCF02F0030EDBCF57
:1005B00003F003500118E8AE02D0013404D000501B
:1005C000025C015003586EE2DECF02F0DDCF03F093
:1005D000D89003320232020EDBCF20F0030EDBCFC5
:1005E00021F00250205C006E03502158016E080E6D
:1005F00000C0DBFF090E01C0DBFFFE0EDB50006E0A
:10060000016AFC0EDB50026E036A0250001802E120
:100610000350011846E0080EDBCF00F0090EDBCFD7
:1006200001F00001800E011416E1FD0EDBCFE7FFA3
:10063000060EDB50E726FD0EE7CFDBFFDECF00F036
:10064000DDCF01F0D950080FE96EDACFEAFF005094
:10065000EE5E0150ED5AFE0EDBCFE7FF040EDB50DD
:10066000E726FE0EE7CFDBFF020EDBCF00F0030E26
:10067000DBCF01F0D950080FE96EDACFEAFF005066
:10068000EE260150ED22FA0EDB50E66EFD0EDB5039
:10069000E66EFE0EDB50E66E2FDEE552E552E552C9
:1006A000ACD769D0020EDBCF02F0030EDBCF03F034
:1006B000D890033202320250DE5C006E0350DD58E7
:1006C000016E080E00C0DBFF090E01C0DBFFFD0E4E
:1006D000DB50006E016AFB0EDB50026E036A0250B3
:1006E000001802E10350011846E0080EDBCF00F0CD
:1006F000090EDBCF01F00001800E011418E1FE0E9F
:10070000DBCFE7FF040EDB50E726FE0EE7CFDBFF73
:10071000020EDBCF00F0030EDBCF01F0D950080F43
:10072000E96EDACFEAFF0050EE5E0150ED5AFD0EA1
:10073000DBCFE7FF060EDB50E726FD0EE7CFDBFF42
:10074000DECF00F0DDCF01F0D950080FE96EDACF2F
:10075000EAFF0050EE260150ED22FA0EDB50E66E65
:10076000FD0EDB50E66EFE0EDB50E66EC5DDE5529B
:10077000E552E552ACD70A0EE15C02E2E16AE552CD
:10078000E16EE552E7CFD9FF1200D9CFE6FFE1CF06
:10079000D9FF020EE126E66AE66A0FDBE552E55272
:1007A00001012D6B2E6BDE6ADD6ADECF00F0DDCF3E
:1007B00001F0000E005C030E015811E2DECFE9FFEC
:1007C000DDCFEAFF830EE926000EEA22EF50E66E47
:1007D000A2DAE552DF2A010E01E3DB2AE6D7020E98
:1007E000E15C02E2E16AE552E16EE552E7CFD9FF52
:1007F0001200D9CFE6FFE1CFD9FFFA0EDB50E66E4B
:10080000FD0EDB50E66EFC0EDB50E66EFD0EDB509F
:10081000E66EFE0EDB50E66E2EDE006E050EE15E2D
:100820000050FA0EDB50E66EFB0EDB50E66EFC0E5F
:10083000DB50E66EFD0EDB50E66EFC0EDB50E66E26
:100840001ADE006E050EE15E0050FA0EDB50E66E19
:10085000FB0EDB50E66EFE0EDB50E66EFB0EDB5051
:10086000E66EFC0EDB50E66E06DE006E050EE15E07
:100870000050FA0EDB50E66EFD0EDB50E66EFE0E0B
:10088000DB50E66EFB0EDB50E66EFE0EDB50E66ED6
:10089000F2DD006E050EE15E005077DFE552E7CF36
:1008A000D9FF1200D9CFE6FFE1CFD9FF050EE1262F
:1008B000030EDB6AFD0EDB50026E036AFE0EDB5098
:1008C000046E056A0450025C006E05500358016E08
:1008D000040E00C0DBFFFC0EDB50E76E020EE7CF1C
:1008E000DBFFFC0EDB50026E036A020E206E216AF3
:1008F00002C025F003C026F01BEC1CF01EC000F067
:100900001FC001F0030ED8800056000E015600C033
:10091000DEFF01C0DDFF030EDB50006E016A020E38
:10092000DB50026E036A03500118E8AE02D00134B6
:1009300004D00050025C0150035801E276D1FB0E56
:10094000DB50E66EFD0EDBCF00F0020EDB50002424
:10095000E66EFE0EDBCF01F0030EDB500124E66EE7
:10096000CBDCE552E552E552FB0EDB50E66EFD0EA8
:10097000DB50026E036A020EDB50046E056A0450FF
:10098000025C006E05500358016E0050E66EFE0ECC
:10099000DBCF06F0030EDB500624E66EADDCE5523D
:1009A000E552E552FB0EDB50E66EFD0EDBCF00F0AC
:1009B000020EDB500024E66EFE0EDB50036E046A6E
:1009C000030EDB50056E066A0550035C016E06508F
:1009D0000458026E0150E66E8FDCE552E552E55296
:1009E000FB0EDB50E66EFD0EDB50026E036A020E5C
:1009F000DB50046E056A0450025C006E055003581B
:100A0000016E0050E66EFE0EDB50086E096A030EA2
:100A1000DB500A6E0B6A0A50085C066E0B500958D0
:100A2000076E0650E66E68DCE552E552E552FB0EB5
:100A3000DB50E66EFD0EDBCF00F0030EDB50002432
:100A4000E66EFD0EDBCF05F0020EDB500524036ED3
:100A5000046A000E0422040EDB50066E076A06507C
:100A6000035C016E07500458026E0150E66E44DCD0
:100A7000E552E552E552FB0EDB50E66EFD0EDB5013
:100A8000026E036A030EDB50046E056A0450025CBA
:100A9000006E05500358016E0050E66EFD0EDBCF70
:100AA0000AF0020EDB500A24086E096A000E0922C1
:100AB000040EDB500B6E0C6A0B50085C066E0C507B
:100AC0000958076E0650E66E17DCE552E552E5520E
:100AD000FB0EDB50E66EFD0EDBCF00F0030EDB50AD
:100AE0000024E66EFD0EDB50056E066A020EDB503A
:100AF000076E086A0750055C036E08500658046EBE
:100B0000040EDB50096E0A6A0950035C016E0A503C
:100B10000458026E0150E66E7CEC01F0E552E5529D
:100B2000E552FB0EDB50E66EFD0EDB50026E036AF3
:100B3000030EDB50046E056A0450025C006E055023
:100B40000358016E0050E66EFD0EDB500A6E0B6A14
:100B5000020EDB500C6E0D6A0C500A5C086E0D50D4
:100B60000B58096E040EDB500E6E0F6A0E50085CB7
:100B7000066E0F500958076E0650E66E7CEC01F0C9
:100B8000E552E552E552DECF00F0DDCF01F0000185
:100B9000800E01141EE0030EDB50026E036A040E89
:100BA000206E216A02C025F003C026F01BEC1CF069
:100BB0001EC000F01FC001F0060E0026000E01222C
:100BC000D9CFE9FFDACFEAFF0050EE260150ED223F
:100BD00029D0030EDB50046E056A020EDB50066E50
:100BE000076A0650045C026E07500558036E040E37
:100BF000206E216A02C025F003C026F01BEC1CF019
:100C00001EC000F01FC001F00A0E0026000E0122D7
:100C1000D9CFE9FFDACFEAFF0050EE260150ED22EE
:100C2000020EDB06030EDB2A76D6AFDD050EE15C95
:100C300002E2E16AE552E16EE552E7CFD9FF120028
:100C4000828282908294960EE66E6EEC01F0E552FE
:100C500082808284640EE66E6EEC01F0E552210E15
:100C6000E66E3FD8E552900EE66E3BD8E552050E93
:100C7000E66E37D8E552130EE66E33D8E552200EF5
:100C8000E66E2FD8E552960EE66E6EEC01F0E55258
:100C90000C0EE66E26D8E552320EE66E6EEC01F0D2
:100CA000E55212008290E66AE66A87D8E552E5527C
:100CB0000001686B696BD890695104E6000E685DAD
:100CC000030E69590DE2E66A26D8E5520A0EE66E71
:100CD00058EC01F0E5520001682B000E6923EBD7B8
:100CE0001200D9CFE6FFE1CFD9FF82928290190E90
:100CF000E66E58EC01F0E552FE0EDBCF00F0016A23
:100D000000BE01680050E66E20D8E5528280E552B0
:100D1000E7CFD9FF1200D9CFE6FFE1CFD9FF82821A
:100D20008290190EE66E58EC01F0E552FE0EDBCF14
:100D300000F0016A00BE01680050E66E06D8E55278
:100D40008280E552E7CFD9FF1200D9CFE6FFE1CF8D
:100D5000D9FFE652080EDF6EDFCF00F0016A00BE59
:100D60000168013404E200500008000E015420E242
:100D700082960A0EE66E58EC01F0E552FE0EDBCFCD
:100D800000F0016A00BE01680050800B02E1829809
:100D900001D082888286FE0EDBCF00F0016A00BEA1
:100DA0000168D8900036013600C0DBFFDF06D4D7DB
:100DB000E552E552E7CFD9FF1200D9CFE6FFE1CFE8
:100DC000D9FFFD0EDB50006E016A070E0016000E03
:100DD0000116400E0010E66E84DFE552FE0EDB5079
:100DE000006E016A7F0E0016000E0116800E0010C4
:100DF000E66E77DFE552E552E7CFD9FF1200D9CF93
:100E0000E6FFE1CFD9FFE652DF6ADFCF00F0016AEB
:100E100000BE0168D890015004E6600E005C000E30
:100E2000015813E2FE0EDB50E66EDFCF00F0016AE0
:100E300000BE01680050E66EC0DFE552E552200EAC
:100E4000E66E83D8E552DF2AE0D7E552E552E7CFD8
:100E5000D9FF1200D9CFE6FFE1CFD9FF020EE1267C
:100E6000E66AE66AAADFE552E552DE6ADD6ADECFAF
:100E700000F0DDCF01F0D890015004E6600E005C78
:100E8000000E01581DE2E66A46DFE552E66A43DFDE
:100E9000E552E66A40DFE552E66A3DDFE552E66A82
:100EA0003ADFE552E66A37DFE552E66A34DFE552BB
:100EB000E66A31DFE552DF2A010E01E3DB2AD7D7EC
:100EC000E66AE66A7ADFE552E552020EE15C02E28A
:100ED000E16AE552E16EE552E7CFD9FF1200D9CFC2
:100EE000E6FFE1CFD9FFE652DF6ADFCF00F0016A0B
:100EF00000BE0168D890015004E6080E005C000EA8
:100F000001581EE2DFCF00F0016A00BE0168005008
:100F1000E66EFE0EDB50E66E50DFE552E552E66A05
:100F2000FADEE552E66AF7DEE552E66AF4DEE552FD
:100F3000E66AF1DEE552E66AEEDEE552DF2AD5D753
:100F4000E552E552E7CFD9FF1200D9CFE6FFE1CF56
:100F5000D9FFFE0EDB5000016A6F6A51006E016A14
:100F6000D890015004E6200E005C000E015801E20A
:100F700075D06A51006E016A013404E200507F08A6
:100F8000000E015401E26AD06B6B6B51006E016A76
:100F9000D890015004E6050E005C000E01585BE29B
:100FA0006A51006E016AD890015004E6500E005C50
:100FB000000E015825E26A51006E016A200E005EA3
:100FC000000E015A050E0102F3CF01F00002F3CF2B
:100FD00000F0F450012600C06CF06B516C25F66EE9
:100FE000F76A000EF722720EF6263B0EF722080073
:100FF000F5CF00F0016A00BE016800C06DF024D09A
:101000006A51006E016A500E005E000E015A050E14
:101010000102F3CF01F00002F3CF00F0F4500126FB
:1010200000C06CF06B516C25F66EF76A000EF7226B
:10103000620EF6263C0EF7220800F5CF00F0016A9A
:1010400000BE016800C06DF06D51E66E64DEE552D1
:1010500000016B2B9AD7E66A5EDEE552E552E7CFD8
:10106000D9FF1200D9CFE6FFE1CFD9FFE652000148
:101070006F6B706B716B726BDF6ADFCF00F0016AB0
:1010800000BE0168FD0EDB50026E036A02500018BC
:1010900002E10350011807E0D8906F3770377137BD
:1010A0007237DF2AEAD76F836FC073F070C074F0B5
:1010B00071C075F072C076F0746B756B766B080E4C
:1010C0001F0B6FC077F070C078F071C079F072C0FC
:1010D0007AF008E00001D8907A33793378337733A7
:1010E000E806F9E10001786B796B7A6B100E1F0B43
:1010F0006FC07BF070C07CF071C07DF072C07EF07C
:1011000008E00001D8907E337D337C337B33E806E2
:10111000F9E100017C6B7D6B7E6B180E1F0B6FC0BD
:101120007FF070C080F071C081F072C082F008E082
:101130000001D8908233813380337F33E806F9E1B0
:101140000001806B816B826B010EE66EFE0EDB5040
:10115000E66E33DEE552E5527FC0E6FF2AD8E5525F
:10116000020EE66EFE0EDB50E66E27DEE552E5521D
:101170007BC0E6FF1ED8E552030EE66EFE0EDB5086
:10118000E66E1BDEE552E55277C0E6FF12D8E55267
:10119000040EE66EFE0EDB50E66E0FDEE552E55203
:1011A00073C0E6FF06D8E552E552E552E7CFD9FF16
:1011B0001200D9CFE6FFE1CFD9FFE65282828290BA
:1011C000080EDF6EDFCF00F0016A00BE0168013457
:1011D00004E200500008000E015420E282960A0E3C
:1011E000E66E58EC01F0E552FE0EDBCF00F0016A2E
:1011F00000BE01680050010B02E1829801D0828894
:101200008286FE0EDBCF00F0016A00BE0168D89036
:101210000132003200C0DBFFDF06D4D78280E55206
:10122000E552E7CFD9FF1200E66AE9DDE552010E8B
:10123000E66EE5DDE552020EE66EE1DDE552030EF7
:10124000E66EDDDDE552040EE66ED9DDE552050EF3
:10125000E66ED5DDE552060EE66ED1DDE552070EEF
:10126000E66ECDDDE5521200D9CFE6FFE1CFD9FF22
:10127000FD0EDB50E66EFE0EDB50E66E9EDDE552A7
:10128000E552200EE66E61DEE552E552E7CFD9FF6A
:101290001200E66A40DDE552040EE66E3CDDE552E2
:1012A000020EE66E38DDE5527F0EE66E34DDE55265
:1012B000020EE66E30DDE552040EE66E2CDDE552E0
:1012C000E66A29DDE552E66A26DDE5521200100ED7
:1012D000E66E21DDE552200EE66E1DDDE5527F0E45
:1012E000E66E19DDE552200EE66E15DDE552100EB4
:1012F000E66E11DDE552E66A0EDDE552E66A0BDDCB
:10130000E552E66A08DDE5521200080EE66E03DDDE
:10131000E5521C0EE66EFFDCE5522A0EE66EFBDCA3
:10132000E552080EE66EF7DCE552080EE66EF3DCD9
:10133000E552F80EE66EEFDCE552E66AECDCE552CB
:10134000E66AE9DCE5521200080EE66EE4DCE552DE
:10135000080EE66EE0DCE5522A0EE66EDCDCE552B5
:101360001C0EE66ED8DCE552080EE66ED4DCE552C3
:10137000E66AD1DCE552E66ACEDCE552E66ACBDC11
:10138000E5521200E66AC7DCE552060EE66EC3DCE3
:10139000E552090EE66EBFDCE552090EE66EBBDCD7
:1013A000E552060EE66EB7DCE552E66AB4DCE552BD
:1013B000E66AB1DCE552E66AAEDCE5521200E66AA6
:1013C000AADCE552060EE66EA6DCE5520F0EE66ECE
:1013D000A2DCE5520F0EE66E9EDCE552060EE66ECE
:1013E0009ADCE552E66A97DCE552E66A94DCE5525F
:1013F000E66A91DCE5521200D9CFE6FFE1CFD9FFD2
:10140000FD0EDBCFE9FFFE0EDBCFEAFFEFCF00F0F2
:10141000016A00BE01680050011013E0FD0EDBCF31
:10142000E9FFDB2AFE0EDBCFEAFF01E3DB2AEFCF89
:1014300000F0016A00BE01680050E66E86DDE552EC
:10144000DFD7E552E7CFD9FF1200DACFE4FFE2CFD2
:10145000DAFFE9CFE4FFEACFE4FFF6CFE4FFF7CF0E
:10146000E4FFF5CFE4FFF3CFE4FFF4CFE4FFFACFDE
:10147000E4FF00EE18F0140EE80403E3EECFE4FFFF
:10148000FBD700EE00F0180EE80403E3EECFE4FF14
:10149000FBD7E652F250020B01E0010E2C6E2D6AD2
:1014A000010E2C1801E12D5022E10001D62B000E77
:1014B000D723D82BD923D42BD5238050080B01E078
:1014C000010E2E6E2F6A2E502F1002E0000E01D05A
:1014D000010E2C6E2D6A2C50E8B08086E8A0809614
:1014E000F2928150D26FD36B010ED26FD36B9E50AC
:1014F000010B2C6E2D6A010E2C1801E12D5061E1BB
:101500000001E22B000EE323050EE25D000EE3591D
:1015100024E3FC51020B01E0010E2C6E2D6A2C50CD
:101520002D1003E1E62B000EE7238050100B01E0A5
:10153000010E2E6E2F6A2E502F1002E0000E01D0E9
:10154000010E2C6E2D6A2C50E8B08088E8A080989F
:10155000E26BE36BE42B000EE5233C0EE45D000E32
:10156000E55926E3DC51D45DDA6FDD51D559DB6FE7
:10157000030E256E266ADAC020F0DBC021F003ECF2
:1015800022F020C0DAF021C0DBF00001DA51DB11DB
:1015900002E1FC8301D0FC93EA51DA25EA6FEB51BA
:1015A000DB21EB6FD4C0DCF0D5C0DDF0E46BE56B84
:1015B000DB0EE66E0B0EE66ED0EC21F0E552E55246
:1015C0009E90E55200EE17F0180EE80403E3E5CF15
:1015D000EDFFFBD700EE2BF0140EE80403E3E5CF9C
:1015E000EDFFFBD7E5CFFAFFE5CFF4FFE5CFF3FF43
:1015F000E5CFF5FFE5CFF7FFE5CFF6FFE5CFEAFF53
:10160000E5CFE9FFE5CFDAFF1100D9CFE6FFE1CF63
:10161000D9FFFE0EDB50A96EA69EA69CA680200ECA
:10162000E66E030EE66EE66AE66A6CEC11F0E552D1
:10163000E552E552E552A85000D0E552E7CFD9FF78
:101640001200D9CFE6FFE1CFD9FFFE0EDB50A96E25
:10165000FD0EDB50A86EA69EA684550EA76EAA0EA0
:10166000A76EA682A150100B01E0010E006E016A68
:101670000050011001E1F6D7A198A694E552E7CFFA
:10168000D9FF1200D9CFE6FFE1CFD9FFFB0EDBCFA8
:10169000E9FFFC0EDBCFEAFFEF50006E016A00505D
:1016A00001101AE0FB0EDBCFE9FFDB2AFC0EDBCFDB
:1016B000EAFF01E3DB2AEF50E66EFD0EDBCF00F020
:1016C000DB2AFE0EDBCF01F001E3DB2A0050E66EE1
:1016D000B8DFE552E552DAD7E552E7CFD9FF12007D
:1016E000D9CFE6FFE1CFD9FF020EE126FD0EDBCF19
:1016F000E6FF8BDFE552DE6EDD6AD9CFE9FFDACF98
:10170000EAFFEE50ED1001E11FD0DFCFE6FF4FEC16
:1017100000F0E552FD0EDB2AFE0E01E3DB2AFD0E92
:10172000DBCF00F0FE0EDBCF01F0013404E200500D
:10173000FF08000E015401E207D0D9CFE9FFDACF4C
:10174000EAFFEE50ED10D2E1E80EE66E030EE66E13
:10175000E66AE66A6CEC11F0E552E552E552E552B4
:10176000020EE15C02E2E16AE552E16EE552E7CF8A
:10177000D9FF1200D9CFE6FFE1CFD9FF0A0EE1264B
:1017800001014D0E5D6F010E5E6FFC0EDBCF00F0B0
:10179000016A00BE0168013404E200500108000E35
:1017A000015401E20CD1FC0EDBCF00F0016A00BE57
:1017B00001680050011028E1FD0EDBCF00F0FE0EA5
:1017C000DBCF01F0060E00C0DBFF070E01C0DBFF20
:1017D000080EDB6A090EDB6A4D0EE66E010EE66E40
:1017E000D950060FE96EDACFEAFFEECFE6FFEECF73
:1017F000E6FFEECFE6FFEFCFE6FF1FEC20F0006E36
:10180000060EE15E005010D04D0EE66E010EE66E43
:10181000FD0EDBCFE6FFFE0EDBCFE6FF85EC1FF013
:10182000E552E552E552E5520001FC51400B01E062
:10183000010E006E016A0050011001E191D04D0EC1
:10184000E66E010EE66E7CEC21F0E552E552020EEA
:10185000F3CFDBFF030EF4CFDBFFDE6ADD6ADECF02
:1018600000F0DDCF01F0020EDBCF02F0030EDBCF84
:1018700003F00250005C0350015831E2020EDBCF4E
:1018800002F0030EDBCF03F0DE50025CE96EDD50A8
:101890000358EA6EE906000EEA5A4D0EE926010EDB
:1018A000EA22EF50E66EFC0EDBCF00F0016A00BECC
:1018B0000168040E0026000E0122DE50005CE96E75
:1018C000DD500158EA6E4D0EE926010EEA22E5527E
:1018D000E750EF6EDF2A010E01E3DB2AC0D7DE6A94
:1018E000DD6ADECF00F0DDCF01F0FC0EDBCF04F0CF
:1018F000056A04BE0568050E0426000E0522020EC8
:10190000DB50045C026E030EDB500558036E025080
:10191000005C0350015824E20001FC51100B01E06F
:10192000010E006E016A005001100BE0DECFE9FFEE
:10193000DDCFEAFF4D0EE926010EEA22300EEF6EF2
:101940000AD0DECFE9FFDDCFEAFF4D0EE926010E1A
:10195000EA22200EEF6EDF2A010E01E3DB2AC1D757
:10196000FC0EDBCFE9FFEA6AE9BEEA68050EE9266C
:10197000000EEA224D0EE926010EEA22EF6A00016E
:10198000FC51800B01E0010E006E016A0050011055
:1019900008E05DC1E6FF5EC1E6FF2EDDE552E552DF
:1019A0000ED05DC1E6FF5EC1E6FFD4EC00F0E5526B
:1019B000E552020EF3CFDBFF030EF4CFDBFF0A0E7E
:1019C000E15C02E2E16AE552E16EE552E7CFD9FF60
:1019D0001200D9CFE6FFE1CFD9FF0E0EE126F90EB6
:1019E000DBCFDEFFDBCFDDFFF80EDBCF02F0036ADB
:1019F00002BE0368033404E202500008000E0354E0
:101A000004E3070E006E016A1BD0F80EDBCF04F072
:101A1000056A04BE0568053404E204501608000E89
:101A2000055404E2170E006E016A0AD0F80EDBCFEF
:101A300000F0016A00BE0168010E0026000E0122BE
:101A4000080E00C0DBFF090E01C0DBFF020EDB6ADF
:101A5000030EDB6AFB0EDBCF00F0FC0EDBCF01F0E8
:101A6000FD0EDBCF02F0FE0EDBCF03F0246A256A09
:101A7000266A276A00C01FF001C020F002C021F0D2
:101A800003C022F0D5EC1CF0010A33E1F90EDBCFE4
:101A9000E9FFDB2AFA0EDBCFEAFF01E3DB2A2D0E9A
:101AA000EF6EFB0EDBCF00F0FC0EDBCF01F0FD0E86
:101AB000DBCF02F0FE0EDBCF03F0246A256A800E36
:101AC000266EBF0E276E00C01FF001C020F002C0BE
:101AD00021F003C022F088EC1BF0FB0E1FC0DBFFDF
:101AE000FC0E20C0DBFFFD0E21C0DBFFFE0E22C07E
:101AF000DBFFFB0EDBCF00F0FC0EDBCF01F0FD0EB9
:101B0000DBCF02F0FE0EDBCF03F0246A256A266AE3
:101B1000276A00C01FF001C020F002C021F003C0FE
:101B200022F0CCEC1CF0010A4AE1FB0EDBCF00F006
:101B3000FC0EDBCF01F0FD0EDBCF02F0FE0EDBCFA3
:101B400003F0246A256A800E266E3F0E276E00C0C1
:101B50001FF001C020F002C021F003C022F0D5EC3C
:101B60001CF0010A2CE1006A016A200E026E410E8F
:101B7000036ED950FB0FE96EFF0EDA20EA6EEECF4E
:101B80001FF0EECF20F0EECF21F0EFCF22F000C01B
:101B900024F001C025F002C026F003C027F088EC35
:101BA0001BF022C0EDFF21C0EDFF20C0EDFF1FC0E4
:101BB000EFFF020EDB06030E01E2DB06B6D7FB0EDB
:101BC000DBCF00F0FC0EDBCF01F0FD0EDBCF02F02F
:101BD000FE0EDBCF03F0246A256A200E266E410E2E
:101BE000276E00C01FF001C020F002C021F003C02A
:101BF00022F0D5EC1CF0010A2EE0FB0EDBCF00F04A
:101C0000FC0EDBCF01F0FD0EDBCF02F0FE0EDBCFD2
:101C100003F0246A256A200E266E410E276E00C04E
:101C20001FF001C020F002C021F003C022F035EC0B
:101C30001BF0FB0E1FC0DBFFFC0E20C0DBFFFD0E08
:101C400021C0DBFFFE0E22C0DBFF020EDB2A030EEB
:101C500001E3DB2AB4D7020EDBCF00F0030EDBCFAB
:101C600001F0D950080FE96EDACFEAFF0050EE26F6
:101C70000150ED22010EF36E040EF3CFDBFF050ED3
:101C8000DB6A040EDBCF20F0050EDBCF21F070EC19
:101C90001AF00A0E1FC0DBFF0B0E20C0DBFF0C0E7C
:101CA00021C0DBFF0D0E22C0DBFF040EDBCF00F0F6
:101CB000050EDBCF01F0080EDBCF02F0090EDBCF03
:101CC00003F001500318E8AE02D0033404D00250F0
:101CD000005C035001582EE20A0EDBCF00F00B0E21
:101CE000DBCF01F00C0EDBCF02F00D0EDBCF03F0EB
:101CF000246A256A200E266E410E276E00C01FF052
:101D000001C020F002C021F003C022F035EC1BF02E
:101D10000A0E1FC0DBFF0B0E20C0DBFF0C0E21C024
:101D2000DBFF0D0E22C0DBFF040EDB2A050E01E3F4
:101D3000DB2ABBD70A0EDBCF04F00B0EDBCF05F09E
:101D40000C0EDBCF06F00D0EDBCF07F0246A256A00
:101D5000266A400E276E04C01FF005C020F006C0A2
:101D600021F007C022F035EC1BF01FC000F020C0AE
:101D700001F021C002F022C003F0D950FB0FE96E40
:101D8000FF0EDA20EA6EEECF1FF0EECF20F0EECF9E
:101D900021F0EFCF22F000C024F001C025F002C0F6
:101DA00026F003C027F09FEC1AF022C0EDFF21C0FF
:101DB000EDFF20C0EDFF1FC0EFFFFB0EDBCF00F0FB
:101DC000FC0EDBCF01F0FD0EDBCF02F0FE0EDBCF11
:101DD00003F0246A256A200E266E410E276E00C08D
:101DE0001FF001C020F002C021F003C022F0D5ECAA
:101DF0001CF0010A13E0FB0EDB6AFC0EDB6A800EAE
:101E0000F36EFD0EF3CFDBFF3F0EF36EFE0EF3CF4E
:101E1000DBFF020EDB2A030E01E3DB2A020EDBCF1F
:101E200000F0030EDBCF01F00001800E01145FE033
:101E3000F90EDBCFE9FFDB2AFA0EDBCFEAFF01E385
:101E4000DB2A300EEF6EF90EDBCFE9FFDB2AFA0E4C
:101E5000DBCFEAFF01E3DB2A2E0EEF6E080EDBCFAD
:101E600000F0090EDBCF01F0800E011414E0020E29
:101E7000DBCF02F0030EDBCF03F0080EDB50025C79
:101E8000006E090EDB500358016E020E00C0DBFF2E
:101E9000030E01C0DBFF040EDB68050EDB68040ED9
:101EA000DBCF00F0050EDBCF01F0020EDBCF02F03E
:101EB000030EDBCF03F003500118E8AE02D001346B
:101EC00004D00050025C0150035811E2F90EDBCF40
:101ED000E9FFDB2AFA0EDBCFEAFF01E3DB2A300E53
:101EE000EF6E040EDB06050E01E2DB06D8D7040E0A
:101EF000DB6A050EDB6A040EDBCF00F0050EDBCFDC
:101F000001F0080EDBCF02F0090EDBCF03F0015029
:101F10000318E8AE02D0033404D00250005C035032
:101F2000015801E3ACD0FB0EDBCF1FF0FC0EDBCF82
:101F300020F0FD0EDBCF21F0FE0EDBCF22F066ECB1
:101F40001CF0060E20C0DBFF070E21C0DBFF300EA9
:101F5000E76E060EDBCF00F0070EDBCF01F0E75097
:101F60000026000E0122F90EDBCFE9FFDB2AFA0E74
:101F7000DBCFEAFF01E3DB2A00C0EFFF040EDBCF7B
:101F800000F0050EDBCF01F0020EDB50001803E17C
:101F9000030EDB5001180BE1F90EDBCFE9FFDB2A62
:101FA000FA0EDBCFEAFF01E3DB2A2E0EEF6E060E00
:101FB000DBCF20F0070EDBCF21F070EC1AF00A0E19
:101FC0001FC0DBFF0B0E20C0DBFF0C0E21C0DBFFB0
:101FD0000D0E22C0DBFF1FC000F020C001F021C0A9
:101FE00002F022C003F0D950FB0FE96EFF0EDA2099
:101FF000EA6EEECF1FF0EECF20F0EECF21F0EFCF64
:1020000022F000C024F001C025F002C026F003C079
:1020100027F09EEC1AF022C0EDFF21C0EDFF20C09A
:10202000EDFF1FC0EFFF006A016A200E026E410E35
:10203000036ED950FB0FE96EFF0EDA20EA6EEECF89
:102040001FF0EECF20F0EECF21F0EFCF22F000C056
:1020500024F001C025F002C026F003C027F088EC70
:102060001BF022C0EDFF21C0EDFF20C0EDFF1FC01F
:10207000EFFF040EDB2A050E01E3DB2A3CD7F90E45
:10208000DBCFE9FFFA0EDBCFEAFFEF6A0E0EE15C71
:1020900002E2E16AE552E16EE552E7CFD9FF1200B4
:1020A000D9CFE6FFE1CFD9FF060EE1260001FC9D66
:1020B000FB0EDBCF1FF0FC0EDBCF20F0FD0EDBCFE5
:1020C00021F0FE0EDBCF22F095EC1CF01EC0DEFFEF
:1020D0001FC0DEFF20C0DEFF21C0DDFFDD52DD526C
:1020E000FB0EDBCF04F0FC0EDBCF05F0FD0EDBCFEB
:1020F00006F0FE0EDBCF07F0F90EDBCF20F0FA0E74
:10210000DBCF21F070EC1AF01FC008F020C009F0FE
:1021100021C00AF022C00BF008C024F009C025F04D
:102120000AC026F00BC027F004C01FF005C020F045
:1021300006C021F007C022F088EC1BF01FC000F0A1
:1021400020C001F021C002F022C003F0F90EDBCF65
:1021500014F0FA0EDBCF15F0166A176A15AE02D02E
:102160001668176814C01EF015C01FF016C020F0C6
:1021700017C021F0DFCF23F0010EDBCF24F0020ED9
:10218000DBCF25F0030EDBCF26F02BEC21F01AC0BD
:1021900010F01BC011F01CC012F01DC013F010C0D5
:1021A0001EF011C01FF012C020F013C021F085EC0A
:1021B0001AF01FC00CF020C00DF021C00EF022C09C
:1021C0000FF00CC024F00DC025F00EC026F00FC09B
:1021D00027F000C01FF001C020F002C021F003C0B2
:1021E00022F09EEC1AF066EC1CF0040E20C0DBFF1F
:1021F000050E21C0DBFF5F0EE66E010EE66ED9CF45
:10220000E9FFDACFEAFFEECFE6FFEECFE6FFEECF53
:10221000E6FFEFCFE6FF1FEC20F0006E060EE15E5A
:1022200000500001FC51800B01E0010E006E016ABC
:102230000050011009E05F0EE66E010EE66EFCEC48
:1022400009F0E552E5520CD05F0EE66E010EE66E27
:10225000D4EC00F0E552E552F3CFC7F0F4CFC8F06C
:102260000001FC51800B01E0010E006E016A00507C
:10227000011006E02E0EE66EA5EC07F0E55205D043
:102280002E0EE66E4FEC00F0E552E66A040EDBCF50
:10229000E6FF050EDBCFE6FFBAEC0BF0E552E552A8
:1022A000E552060EE15C02E2E16AE552E16EE552BA
:1022B000E7CFD9FF12008168030E936E938093825B
:1022C000C26A070EC16E926E896A7F0E8B6E800E97
:1022D000946E948E949C1200D9CFE6FFE1CFD9FF83
:1022E000FB0EDBCF1FF0FC0EDBCF20F0FD0EDBCFB3
:1022F00021F0FE0EDBCF22F02234000E221809E678
:10230000D880000E1F54000E2054000E2154000EE1
:1023100022540CE2D950FB0FE96EFF0EDA20EA6E70
:10232000EE06000EEE5AEE5AEE5ADAD7E552E7CF35
:10233000D9FF1200C0DF808680880001FC9BFC8DE5
:10234000FC8FFC99000E626F010E636F62C060F03B
:1023500063C061F001015F0E9F6F010EA06F16EC6C
:1023600000F00C0EE66E4FEC00F0E552500EE66EFB
:10237000C30EE66EE66AE66AAFDFE552E552E55265
:10238000E55211EC01F09FC1E6FFA0C1E6FFD4ECDD
:1023900000F0E552E552F3CFC7F0F4CFC8F011ECEE
:1023A00001F0A4C100F0A5C101F0026A00C0E6FF7F
:1023B00001C0E6FF02C0E6FF5F0EE66E010EE66EAC
:1023C00063EC21F0036E050EE15E03505F0EE66ED6
:1023D000010EE66ED4EC00F0E552E552F3CFC7F003
:1023E000F4CFC8F011EC01F0B0C100F0B1C101F0C0
:1023F000026A00C0E6FF01C0E6FF02C0E6FF5F0E12
:10240000E66E010EE66E63EC21F0036E050EE15EF2
:1024100003505F0EE66E010EE66ED4EC00F0E5525E
:10242000E552F3CFC7F0F4CFC8F011EC01F0000E85
:10243000E66EE66A70EC0BF0E552E55211EC01F045
:10244000200EE66EE66A70EC0BF0E552E55211ECF8
:1024500001F0400EE66EE66A70EC0BF0E552E552D4
:1024600011EC01F0600EE66EE66A70EC0BF0E552DE
:10247000E55211EC01F0800EE66EE66A70EC0BF0AE
:10248000E552E55211EC01F0A00EE66EE66A70EC42
:102490000BF0E552E55211EC01F0C00EE66EE66A73
:1024A00070EC0BF0E552E55211EC01F0E00EE66E37
:1024B000E66A70EC0BF0E552E55211EC01F011EC1C
:1024C00001F00001FC9BFC8DFC8F20EC06F0100E4F
:1024D000E66E270EE66EE66AE66AFEDEE552E55235
:1024E000E552E55280962AEC07F00001FC8FC36BA1
:1024F000C46B070EC35D000EC45937E2C3C0E6FFCC
:10250000E66ADDEC06F0E552E552C3C0E9FFC4C05F
:10251000EAFF010ED890E936EA36E806FBE1B20E92
:10252000E926010EEA22EECF00F0EFCF01F0026AB9
:1025300000C0E6FF01C0E6FF02C0E6FF5F0EE66EE8
:10254000010EE66E63EC21F0036E050EE15E0350B2
:102550005F0EE66E010EE66EFCEC09F0E552E55208
:102560000001C32B000EC423C4D7C36BC46B8050BF
:10257000080B01E0010E026E036A0250031002E034
:10258000000E01D0010E006E016A0050E8B0808696
:10259000E8A08096070EE66EE66ADDEC06F0E552EE
:1025A000E552C8C100F0C9C101F0026A00C0E6FFEF
:1025B00001C0E6FF02C0E6FF5F0EE66E010EE66EAA
:1025C00063EC21F0036E050EE15E03505F0EE66ED4
:1025D000010EE66EFCEC09F0E552E552300EE66EB7
:1025E000750EE66EE66AE66A77DEE552E552E5527A
:1025F000E552070EE66EE66ADDEC06F0E552E552BE
:10260000CAC100F0CBC101F0026A00C0E6FF01C000
:10261000E6FF02C0E6FF5F0EE66E010EE66E63ECBB
:1026200021F0036E050EE15E03505F0EE66E010EB3
:10263000E66EFCEC09F0E552E552300EE66E750EE2
:10264000E66EE66AE66A48DEE552E552E552E55294
:102650000001C32B000EC423030EC35D000EC4593A
:1026600001E285D7070EE66EE66ADDEC06F0E5527C
:10267000E552CCC100F0CDC101F0026A00C0E6FF16
:1026800001C0E6FF02C0E6FF5F0EE66E010EE66ED9
:1026900063EC21F0036E050EE15E03505F0EE66E03
:1026A000010EE66EFCEC09F0E552E552300EE66EE6
:1026B000750EE66EE66AE66A0FDEE552E552E55211
:1026C000E5520001D26BD36BE06BE16BDE6BDF6B2D
:1026D000D66BD76BD86BD96BD46BD56BDA6BDB6BE6
:1026E000DC6BDD6BEA6BEB6BE86BE96BEC6BED6B5A
:1026F000EE6BEF6BE66BE76B7C0EE66E8AEC21F01F
:10270000E552F292F288750EE66EAFEC21F0E552DA
:10271000CD92CD8E9F80D08EDB0EE66E0B0EE66ED8
:10272000D0EC21F0E552E5529E90F28CCD909D8048
:10273000F28EF28C0001FC8FD251D311FDE0D26BEE
:10274000D36BE26BE36BE46BE56BE66BE76B070E59
:10275000E66EE66ADDEC06F0E552E552CEC100F029
:10276000CFC101F0026A00C0E6FF01C0E6FF02C06F
:10277000E6FF5F0EE66E010EE66E63EC21F0036E7F
:10278000050EE15E03505F0EE66E010EE66EFCEC98
:1027900009F0E552E5528086CD800001FC81FC9372
:1027A0000001010ED21901E1D35101E02CD22A0E11
:1027B000D880D655000ED7550FE2D66BD76BE02BDD
:1027C000000EE123E82BE923090ED880E055000E26
:1027D000E15502E2E06BE16BA40ED880D855010E02
:1027E000D9550BE2D86BD96BDE2B000EDF23E82B1B
:1027F000E923E06BE16BD66BD76BFC8DFC8F020E8F
:10280000E66E310EE66EDDEC06F0E552E552E66A64
:10281000D4C0E6FFD5C0E6FFBAEC0BF0E552E552B6
:10282000E552030EE66E310EE66EDDEC06F0E55283
:10283000E552E66ADAC0E6FFDBC0E6FFBAEC0BF071
:10284000E552E552E552040EE66E230EE66EDDEC2F
:1028500006F0E552E552E66ADEC0E6FFDFC0E6FFBD
:10286000BAEC0BF0E552E552E5522E0EE66EA5EC01
:1028700007F0E552300E0001E025E66EA5EC07F00A
:10288000E55200013C0EE65D000EE75942E2060EFD
:10289000E66E1C0EE66EDDEC06F0E552E552E6C093
:1028A00000F0E7C001F00001016A010E00160050BF
:1028B000011015E0570EE66EA5EC07F0E552610E2B
:1028C000E66EA5EC07F0E552690EE66EA5EC07F0A2
:1028D000E552740EE66EA5EC07F0E55214D0200E1A
:1028E000E66EA5EC07F0E552200EE66EA5EC07F0CB
:1028F000E552200EE66EA5EC07F0E552200EE66EDE
:10290000A5EC07F0E5520001EC6BED6BEE6BEF6BA5
:102910006ED0060EE66E1C0EE66EDDEC06F0E5529D
:10292000E552D4C020F0D5C021F06EEC1AF01FC0E3
:1029300004F020C005F021C006F022C007F08C0E84
:10294000246E390E256E090E266E410E276E04C0C8
:102950001FF005C020F006C021F007C022F088EC6F
:102960001BF01FC000F020C001F021C002F022C007
:1029700003F0E6C020F0E7C021F06EEC1AF01FC0B3
:1029800008F020C009F021C00AF022C00BF008C0F6
:1029900024F009C025F00AC026F00BC027F000C0C3
:1029A0001FF001C020F002C021F003C022F035EC7E
:1029B0001BF01FC0ECF020C0EDF021C0EEF022C0F3
:1029C000EFF0640EE66EE66AECC0E6FFEDC0E6FFEF
:1029D000EEC0E6FFEFC0E6FF50EC10F0006E060E12
:1029E000E15E0050090EE66E4FEC00F0E5528150BA
:1029F000020B01E0010E006E016A0050011001E1BE
:102A000002D10001FC9FFC8D4B0EE66E4FEC00F0F6
:102A1000E5526D0EE66E4FEC00F0E552730EE66E79
:102A20004FEC00F0E5523D0EE66E4FEC00F0E55243
:102A3000E66ADEC0E6FFDFC0E6FFBAEC0BF0E55267
:102A4000E552E5522E0EE66E4FEC00F0E552300EE8
:102A50000001E025E66E4FEC00F0E552090EE66E4F
:102A60004FEC00F0E552E66AE6C0E6FFE7C0E6FF9D
:102A7000BAEC0BF0E552E552E552090EE66E4FEC6A
:102A800000F0E552E66AD4C0E6FFD5C0E6FFBAEC36
:102A90000BF0E552E552E55200013C0EE65D000EFA
:102AA000E7591FE2200EE66E4FEC00F0E552570E9C
:102AB000E66E4FEC00F0E552610EE66E4FEC00F072
:102AC000E552690EE66E4FEC00F0E552740EE66ECC
:102AD0004FEC00F0E5520001EC6BED6BEE6BEF6B31
:102AE0008ED0090EE66E4FEC00F0E552E66ADAC0D1
:102AF000E6FFDBC0E6FFBAEC0BF0E552E552E5522B
:102B0000D4C020F0D5C021F06EEC1AF01FC004F044
:102B100020C005F021C006F022C007F08C0E246E04
:102B2000390E256E090E266E410E276E04C01FF069
:102B300005C020F006C021F007C022F088EC1BF091
:102B40001FC000F020C001F021C002F022C003F03D
:102B5000E6C020F0E7C021F06EEC1AF01FC008F0CC
:102B600020C009F021C00AF022C00BF008C024F0F8
:102B700009C025F00AC026F00BC027F000C01FF0E6
:102B800001C020F002C021F003C022F035EC1BF0A0
:102B90001FC0ECF020C0EDF021C0EEF022C0EFF03D
:102BA000090EE66E4FEC00F0E5524D0EE66E4FEC6E
:102BB00000F0E5526F0EE66E4FEC00F0E552790E34
:102BC000E66E4FEC00F0E5523D0EE66E4FEC00F085
:102BD000E552640EE66EE66AECC0E6FFEDC0E6FF85
:102BE000EEC0E6FFEFC0E6FF50EC10F0006E060E00
:102BF000E15E0050090EE66E4FEC00F0E552000178
:102C0000FC8D11EC01F00001D26BD36BFC8F050E33
:102C1000E66E310EE66EDDEC06F0E552E552E66A50
:102C2000E6C0E6FFE7C0E6FFBAEC0BF0E552E5527E
:102C3000E5528050020B01E0010E006E016A010EA8
:102C4000001801E1015001E1ABD5F29CCD909D90BF
:102C5000F29EF29C070EE66EE66ADDEC06F0E552A7
:102C6000E552D0C100F0D1C101F0026A00C0E6FF18
:102C700001C0E6FF02C0E6FF5F0EE66E010EE66EE3
:102C800063EC21F0036E050EE15E03505F0EE66E0D
:102C9000010EE66EFCEC09F0E552E552100EE66E10
:102CA000270EE66EE66AE66A6CEC11F0E552E55234
:102CB000E552E5520001FC9FFC99FC9DA80EE66ED2
:102CC000610EE66EE66AE66A6CEC11F0E552E552DA
:102CD000E552E55211EC01F04B0EE66E4FEC00F0C0
:102CE000E5526D0EE66E4FEC00F0E552730EE66EA7
:102CF0004FEC00F0E5523D0EE66E4FEC00F0E55271
:102D0000E66ADEC0E6FFDFC0E6FFBAEC0BF0E55294
:102D1000E552E5522E0EE66E4FEC00F0E552300E15
:102D20000001E025E66E4FEC00F0E55211EC01F0F9
:102D3000E66AE8C0E6FFE9C0E6FFBAEC0BF0E55250
:102D4000E552E55211EC01F0E66ADAC0E6FFDBC0BD
:102D5000E6FFBAEC0BF0E552E552E55211EC01F05A
:102D6000E66AD4C0E6FFD5C0E6FFBAEC0BF0E55248
:102D7000E552E55211EC01F0E66AE6C0E6FFE7C075
:102D8000E6FFBAEC0BF0E552E552E55211EC01F02A
:102D900000013C0ED880E655000EE75551E2D4C044
:102DA00020F0D5C021F06EEC1AF01FC004F020C056
:102DB00005F021C006F022C007F08C0E246E390EFB
:102DC000256E090E266E410E276E04C01FF005C049
:102DD00020F006C021F007C022F088EC1BF01FC0D5
:102DE00000F020C001F021C002F022C003F0E6C0D4
:102DF00020F0E7C021F06EEC1AF01FC008F020C0F0
:102E000009F021C00AF022C00BF008C024F009C06C
:102E100025F00AC026F00BC027F000C01FF001C04B
:102E200020F002C021F003C022F035EC1BF01FC0DF
:102E3000ECF020C0EDF021C0EEF022C0EFF004D0A5
:102E4000EC6BED6BEE6BEF6B010EE66E2F0EE66E2C
:102E5000010EE66EECC0E6FFEDC0E6FFEEC0E6FF59
:102E6000EFC0E6FFE9EC0CF0006E070EE15E0050EB
:102E70002F0EE66E010EE66E7CEC21F0E552E55277
:102E8000F3CF00F0F4CF01F0050ED8800054000E0F
:102E9000015402E20101346B2F0EE66E010EE66E64
:102EA000D4EC00F0E552E55211EC01F011EC01F028
:102EB000010E0001D06FD16BC36FC46B090EC35DEF
:102EC000000EC45926E2C3C0C7F0C4C0C8F0010E4A
:102ED000C75F000EC85B050ED890C737C837E80635
:102EE000FBE1C7C0E6FF05EC0BF0E5520001CB6F3C
:102EF000CB51006E016A300E001801E1015005E16E
:102F0000C3C0D0F0C4C0D1F004D0C32B000EC42382
:102F1000D5D7070ED880C355000EC45508E2300E31
:102F2000E66EE66A21EC0BF0E552E55215D0200E74
:102F3000206E216AC3C025F0C4C026F048EC1CF006
:102F40001EC0C7F01FC0C8F0300EE66EC7C0E6FF57
:102F500021EC0BF0E552E5520001FC99FC8DB4C167
:102F600000F0B5C101F0026A00C0E6FF01C0E6FF53
:102F700002C0E6FF5F0EE66E010EE66E63EC21F026
:102F8000036E050EE15E03505F0EE66E010EE66E07
:102F9000D4EC00F0E552E552F3CFC7F0F4CFC8F01F
:102FA000E66AD0C0E6FFD1C0E6FFBAEC0BF0E5520E
:102FB000E552E552090EE66E4FEC00F0E552D0C046
:102FC000C7F0D1C0C8F00001010EC75F000EC85B9A
:102FD000050ED890C737C837E806FBE1300E000170
:102FE000D025E66EC7C0E6FF21EC0BF0E552E552B6
:102FF000C7C0D0F0C8C0D1F0E66AD0C0E6FFD1C0EB
:10300000E6FFBAEC0BF0E552E552E55211EC01F0A7
:103010000001D02B000ED1233B0EE66ED0C0E6FFA0
:1030200021EC0BF0E552E5520001D02B000ED1232C
:1030300001014D0E5D6F010E5E6FE66ADAC0E6FFBC
:10304000DBC0E6FFBAEC0BF0E552E552E552090EA3
:10305000E66E4FEC00F0E5520001C36BC46B050E49
:10306000C35D000EC45915E24D0EC325E96E010E75
:10307000C421EA6EEF50E66ED0C0E6FF21EC0BF003
:10308000E552E5520001D02B000ED123C32BC423FF
:10309000E6D73B0EE66ED0C0E6FF21EC0BF0E55222
:1030A000E5520001D02B000ED12301014D0E5D6FC2
:1030B000010E5E6FE66AE6C0E6FFE7C0E6FFBAEC27
:1030C0000BF0E552E552E552090EE66E4FEC00F0CA
:1030D000E5520001C36BC46B050EC35D000EC459FD
:1030E00015E24D0EC325E96E010EC421EA6EEF50C4
:1030F000E66ED0C0E6FF21EC0BF0E552E552000190
:10310000D02B000ED123C32BC423E6D73B0EE66E93
:10311000D0C0E6FF21EC0BF0E552E5520001D02BC8
:10312000000ED12301014D0E5D6F010E5E6FE66A48
:10313000E8C0E6FFE9C0E6FFBAEC0BF0E552E55265
:10314000E552090EE66E4FEC00F0E5520001C36B4C
:10315000C46B050EC35D000EC45915E24D0EC325A8
:10316000E96E010EC421EA6EEF50E66ED0C0E6FFB4
:1031700021EC0BF0E552E5520001D02B000ED123DB
:10318000C32BC423E6D73B0EE66ED0C0E6FF21EC8E
:103190000BF0E552E5520001D02B000ED1230101C6
:1031A0004D0E5D6F010E5E6FE66AD4C0E6FFD5C0BE
:1031B000E6FFBAEC0BF0E552E552E5520001C36BB5
:1031C000C46B050EC35D000EC45915E24D0EC32538
:1031D000E96E010EC421EA6EEF50E66ED0C0E6FF44
:1031E00021EC0BF0E552E5520001D02B000ED1236B
:1031F000C32BC423E6D73B0EE66ED0C0E6FF21EC1E
:103200000BF0E552E5520001D02B000ED1233D0E0C
:10321000E65D000EE75904E2EC6BED6BEE6BEF6BD5
:10322000010EE66E2F0EE66E010EE66EECC0E6FFB6
:10323000EDC0E6FFEEC0E6FFEFC0E6FFE9EC0CF004
:10324000006E070EE15E00502F0EE66E010EE66E78
:103250007CEC21F0E552E552F3CF00F0F4CF01F021
:10326000050ED8800054000E015402E20101346BB7
:10327000020EE66E2F0EE66E010EE66EECC0E6FF65
:10328000EDC0E6FFEEC0E6FFEFC0E6FFE9EC0CF0B4
:10329000006E070EE15E005011EC01F02F0EE66E9D
:1032A000010EE66E7CEC21F0E552E552F3CFC7F05B
:1032B000F4CFC8F00001050ED880C755000EC855E0
:1032C00005E2050EC76FC86B0101346B0001C36BCB
:1032D000C46BC751C35DC851C45915E22F0EC32535
:1032E000E96E010EC421EA6EEF50E66ED0C0E6FF33
:1032F00021EC0BF0E552E5520001D02B000ED1235A
:10330000C32BC423E6D711EC01F0F00EE66E490E94
:10331000E66E020EE66EE66A6CEC11F0E552E552DE
:10332000E552E55211EC01F0B0C100F0B1C101F07D
:10333000026A00C0E6FF01C0E6FF02C0E6FF5F0EC2
:10334000E66E010EE66E63EC21F0036E050EE15EA3
:1033500003505F0EE66E010EE66ED4EC00F0E5520F
:10336000E552F3CFC7F0F4CFC8F011EC01F0E80E4E
:10337000E66E030EE66EE66AE66A6CEC11F0E55264
:10338000E552E552E5520001C56BC66BFF0EC55D07
:10339000000EC6593CE2C36BC46B200EC35D000E29
:1033A000C4592BE2C551C325E66E05EC0BF0E5527E
:1033B0000001CB6FCB51006E016AD890015004E63A
:1033C000200E005C000E015802E22E0ECB6FCB5196
:1033D000E66E4FEC00F0E552E80EE66E030EE66E88
:1033E000E66AE66A6CEC11F0E552E552E552E55208
:1033F0000001C32B000EC423D0D711EC01F0200E26
:103400000001C525C56F000EC621C66FBFD711ECE0
:1034100001F011EC01F0A8C100F0A9C101F0026AAD
:1034200000C0E6FF01C0E6FF02C0E6FF5F0EE66EE9
:10343000010EE66E63EC21F0036E050EE15E0350B3
:103440005F0EE66E010EE66ED4EC00F0E552E5523A
:10345000F3CFC7F0F4CFC8F011EC01F08050100B9F
:1034600001E0010E026E036A0250031002E0000E3A
:1034700001D0010E006E016A0050E8B08088E8A01B
:103480008098E80EE66E030EE66EE66AE66A6CEC7D
:1034900011F0E552E552E552E5528050080B01E08B
:1034A000010E026E036A0250031002E0000E01D00A
:1034B000010E006E016A0050E8B08086E8A0809698
:1034C000E80EE66E030EE66EE66AE66A6CEC11F054
:0C34D000E552E552E552E552C1D712006A
:0434DC00199E08D05D
:1034E000199E21AE05D0206C211EE86A2122198E7A
:1034F00021C01BF020C01AF02B6A2A6A8E0E1C6EA7
:103500001D6A4FEF1DF0199E0CD0199E21AE09D0F7
:103510001E6C1F1E201E211EE86A1F22202221224F
:10352000198E21C01BF020C01AF01FC02BF01EC046
:103530002AF09E0E1C6E1D6A4FEF1DF0277E196A41
:103540008BEC1DF0A3EC1DF019B633EF1DF019A2A2
:103550000AD019AA03D019BE33EF1DF019A43FEF0A
:103560001DF03CEF1DF019AA05D019AC3FEF1DF07E
:103570003CEF1DF019A00AD019A808D019BE04D03C
:1035800019A402D048EF1DF04CEF1DF02A6A1D6A05
:103590002750225C296E10E31FC02BF020C01AF0C8
:1035A00021C01BF022C028F024C01FF025C020F04D
:1035B00026C021F0193A09D024C02BF025C01AF0FA
:1035C00026C01BF027C028F0296C199E19BC198E43
:1035D00028C01CF019B07BEF1DF01A0E29607BEF9C
:1035E0001DF01C6A226A19A408D01F6C201E211E1F
:1035F000221EE86A20222122222219AC08D02B6C3C
:103600001A1E1B1E1C1EE86A1A221B221C221E6A7E
:10361000295207E02234213220321F321E32292E55
:10362000F9D71F502B2620501A2221501B2222503E
:103630001C221EC02AF0199E1CAE0BD02A6C2B1E19
:103640001A1E1B1E1C1EE86A2B221A221B221C2279
:10365000198E1CA006D0D8801B321A322B322A3287
:10366000282A28C01CF04FEF1DF0196A8BEC1DF0C2
:10367000A3EC1DF019B633EF1DF019A205D019BA4D
:1036800033EF1DF03AEF1DF019BA46EF1DF019A007
:1036900005D019B833EF1DF046EF1DF019B83AEF19
:1036A0001DF01D6A7F0E22241C6EE86A1D22275021
:1036B0001C5EE86A1D5A1A0E286E226A2A6A2B6A54
:1036C0001A6A1B6A24501F5E2550205A2650215A20
:1036D000000E225A09E724501F262550202226508A
:1036E0002122000E222201D02A8AD8901F362036AD
:1036F00021362236D8902A362B361A361B36282EFB
:10370000E1D7215020101F10D8A42A8A4FEF1DF0B6
:10371000196A8BEC1DF0A3EC1DF019B633EF1DF008
:1037200019A205D019B833EF1DF03AEF1DF019AA10
:1037300005D019B033EF1DF03AEF1DF019B002D0EB
:1037400019A802D046EF1DF01D6A275022241C6ED6
:10375000E86A1D227E0E1C5EE86A1D5A2A6A2B6AE0
:103760001A6A1B6A26502102F4CF1BF0F3CF1AF01D
:1037700025502102F3502B26F4501A22000E1B2252
:1037800026502002F3502B26F4501A22000E1B2242
:1037900024502102F3502A26F4502B22000E1A2224
:1037A0001B2225502002F3502A26F4502B22000E13
:1037B0001A221B2226501F02F3502A26F4502B22D5
:1037C000000E1A221B2224502002F4502A26000E3A
:1037D0002B221A221B2225501F02F4502A26000EEB
:1037E0002B221A221B224FEF1DF0186A26AEFEEF85
:1037F0001BF0256C261EE86A2622181E21AE06EF55
:103800001CF0206C211EE86A2122181E03EC22F015
:1038100021BE16EF1CF018AE000C206C211EE86AC9
:1038200021221C6C1D1EE86A1D22000C18BE0DEF23
:103830001CF01988FF0C21C02BF020C02AF020506A
:103840002502F4CF1FF0F3CF1EF021502602F4CF53
:1038500021F0F3CF20F02502F3501F26F450202250
:10386000E86A21222A502602F3501F26F450202213
:10387000E86A212226AE41EF1CF02A50205E2B5030
:10388000215A2BAE000C2550205E2650215A000CE8
:1038900020C02AF020502502F4CF1FF0F3CF1EF0F5
:1038A00021502602F4CF21F0F3CF20F02502F3506F
:1038B0001F26F4502022E86A21222A502602F350C3
:1038C0001F26F4502022E86A2122000C196A8BEC92
:1038D0001DF019B670EF1CF019A20ED019B405D066
:1038E0007F0E216EFF0E206E1FD0800E216E206A8B
:1038F0001BD0216A206A18D019B0FBD78F0E226026
:10390000EDD77E0E2264F5D78E0E225C05E0D890AE
:1039100021322032222AF8D719A406D0206C211E89
:10392000E86A212221AEE5D71200196A8BEC1DF05E
:1039300019B69FEF1CF019A20FD019B407D07F0E53
:10394000216EFF0E206E1F6E1E6E25D0800E216E22
:1039500001D0216A000EF6D719B0FBD71E6A9F0E60
:103960002260EBD77E0E2264F4D79E0E225C07E025
:10397000D890213220321F321E32222AF6D719A4C3
:103980000AD01E6C1F1E201E211EE86A1F22202244
:10399000212221AEDED71200DEEC1CF019B6000C9D
:1039A00019B0000C19B4000C010CDEEC1CF019B6B7
:1039B000000C19B0000C19A4000C010C196A8BEC56
:1039C0001DF0A3EC1DF019B6120019AE08D019A015
:1039D00004D019A802D019801200199012002750A3
:1039E000225C0BE12650215C08E12550205C05E1BA
:1039F00024501F5C02E119801200D8A002D0198E59
:103A000010D0225027C022F0276E215026C021F06E
:103A1000266E205025C020F0256E1F5024C01FF0B8
:103A2000246E2750225C10E0FF0F09E0199019B4B2
:103A300003D019AE1984120019AE19941200272A66
:103A4000D89026322532243224501F5E2550205A29
:103A50002650215A21BEEAD7D8901F36203621366B
:103A6000222EF8D7C8D77F0E226EFF0E216E206E51
:103A70001F6E12007F0E19BEFF0E226E02D07F0E47
:103A8000226E800E216E206A1F6AF3D719AE04D011
:103A9000800E226E216AF7D7226A216AF4D71B5062
:103AA0001A102B102A10F8E01DBEF0D71BBE0CD048
:103AB0001C501D10EBE0D8902A362B361A361B36D8
:103AC0001C06D8A01D06F2D71D50D4E11C28D2E058
:103AD0002AAE11D07F0E2A1402E12BA00CD02B2A83
:103AE000E86A1A221B2207E3D8801B321A322B32D3
:103AF0001C2A1C28BFE01C50C9E02BC01FF01AC0B4
:103B000020F01B34216E1C30226E2132229E19BE01
:103B1000228E39EF1DF02136223602E31984197EF8
:103B200006E11980226A216A206A1F6A120022288F
:103B300003E0D88021321200D890213202E11982AC
:103B40001200198612002636273602E3198C197ED8
:103B500006E11988276A266A256A246A120027283E
:103B600003E0D88026321200D8902632EAE1198A82
:023B7000120041
:0E3B7200000000000000005F000000070007D8
:103B800000147F147F14242A7F2A122313086462EE
:103B900036495522500005030000001C2241000058
:103BA00041221C0014083E081408083E0808005072
:103BB00030000008080808080060600000201008B5
:103BC00004023E5149453E00427F40004261514956
:103BD000462141454B311814127F10274545453980
:103BE0003C4A4949300171090503364949493606BD
:103BF0004949291E003636000000563600000814D8
:103C0000224100141414141400412214080201511A
:103C10000906324979413E7E1111117E7F49494999
:103C2000363E414141227F4141221C7F4949494161
:103C30007F090909013E4149497A7F0808087F0048
:103C4000417F41002040413F017F081422417F40D5
:103C50004040407F020C027F7F0408107F3E4141BC
:103C6000413E7F090909063E4151215E7F0919291C
:103C700046464949493101017F01013F4040403FEB
:103C80001F2040201F3F4038403F63140814630743
:103C9000087008076151494543007F414100020413
:103CA0000810200041417F0004020102044040400E
:103CB0004040000102040020545454787F4844449A
:103CC000383844444420384444487F3854545418C5
:103CD000087E0901020C5252523E7F08040478000B
:103CE000447D40002040443D007F102844000041B6
:103CF0007F40007C041804787C080404783844442D
:103D000044387C14141408081414187C7C08040427
:103D1000084854545420043F4440203C4040207CF8
:103D20001C2040201C3C4030403C44281028440CBF
:103D30005050503C4464544C44000836410000004C
:103D40007F0000004136080010080810087846413E
:103D50004678506F727420636F6D6D203139323048
:103D600030206F75766572740A004331383A313805
:103D7000463235385F56656C6F5F4E6F6B69615FB9
:103D80003131303930312E63200D0A004553432044
:103D9000706F757220736F727469720D0A00536FC1
:103DA00072746965204E6F726D616C652064652068
:103DB000507267004170707579657220737572205A
:103DC00042502053746172740D004F6E20726F75F3
:103DD0006C65202E2E2E0D00417070756920737554
:103DE000722042502053746F700D0023204E627475
:103DF00064503B5365633B686563744D3B5464504A
:103E00002F4D3B564D6F790031383235382056658D
:103E10006C6F204E6F6B696100506172636F7572D9
:103E20007320232020202020004E6250756C733AAE
:103E30002020202020202020004E627464702F4D0E
:103E40006E3A2020202020200044697374616E6344
:103E50003A20202020204B6D0044757265653A2081
:103E60002020202020202053004D6F793A20202050
:103E7000202020204B6D2F4800202E2E2E2E2E2E5F
:103E80002E2E2E2E2E2E2E200044752E546F743A78
:103E9000202020202E20204800546450544F543AB3
:103EA0002020202020202020004E624B6D735420C3
:103EB0003A20202020202020004170707569207356
:103EC000757220535441525400202020202020207D
:103ED0002020202020202020002E2E2E2E53746102
:103EE0007274696E672E2E20002E2E2052756E6E13
:103EF000696E67202E2E2E200020536F7274696524
:093F0000202F2053544F502000E3
:063F0A00D9CFE6FFDACF7B
:103F1000E6FFFA0EE3CFD9FFFB0EE3CFDAFFFD0E8B
:103F2000E35209E72D0EDE6EFC0EE31EE32AFD0EC2
:103F3000D8B4E306E31EE652E652E652FD0EE12453
:103F4000E76EFF0EE220E46EE652F70EE3CFE6FFE7
:103F5000F70EE3CFE6FFF5EC1FF0F90EE124E96E72
:103F6000FF0EE220EA6EE5EC1FF00AE1E2EC1FF042
:103F700009E1E5EC1FF008E1E2EC1FF007E108D0F1
:103F8000F0EC1FF0EBEC1FF0F0EC1FF0EBEC1FF08F
:103F9000F0EC1FF0DE6AF90EE126FF0EE222FF0EC2
:103FA000E3CFDAFFE552FF0EE3CFD9FFE552FC0E77
:103FB000E124E96EFF0EE220EA6EEECFF3FFEFCFD1
:103FC000F4FF1200EF380F0B1200EF500F0B02E15D
:103FD000EE52D8841200EF380F0B300FDE6E120055
:103FE000EE500F0B300FDE6E1200FC0EE3CFE9FF38
:103FF000FD0EE3CFEAFF100EE66EEE6AEE6AEF6AA0
:10400000D890FD0EE336FE0EE336ED36ED36EF3694
:10401000FF0EE30609E016EC20F0EE5216EC20F05D
:10402000EE5216EC20F0EDD7E56E1200030EEF24F1
:10403000E8B6EF6E300EEF24E8BEEF6E000CD9CF7D
:10404000E6FFDACFE6FFF80EE3CFD9FFF90EE3CFB4
:10405000DAFFE652E652E652E652E652FB0EE12461
:10406000E76EFF0EE220E46EE652F30EE3CFE6FFCA
:10407000F30EE3CFE6FFF30EE3CFE6FFF30EE3CF5D
:10408000E6FFA4EC20F0F50EE124E96EFF0EE2203D
:10409000EA6E91EC20F019E194EC20F018E191EC3B
:1040A00020F017E194EC20F016E191EC20F015E1FE
:1040B00094EC20F014E191EC20F013E194EC20F06A
:1040C00012E191EC20F011E112D09AEC20F09FEC7B
:1040D00020F09AEC20F09FEC20F09AEC20F09FEC7E
:1040E00020F09AEC20F09FEC20F09AEC20F09FEC6E
:1040F00020F0DE6AF50EE126FF0EE222FF0EE3CF8E
:10410000DAFFE552FF0EE3CFD9FFE552FA0EE124C4
:10411000E96EFF0EE220EA6EEECFF3FFEFCFF4FF81
:104120001200EF380F0B1200EF500F0B02E1EE52AE
:10413000D8841200EF380F0B300FDE6E1200EE50F5
:104140000F0B300FDE6E1200FA0EE3CFE9FFFB0E0D
:10415000E3CFEAFF200EE66EEE6AEE6AEE6AEE6AE2
:10416000EF6AD890FB0EE336FC0EE336FD0EE33625
:10417000FE0EE336ED36ED36ED36ED36EF36FF0E5C
:10418000E3060FE0D3EC20F0EE52D3EC20F0EE5239
:10419000D3EC20F0EE52D3EC20F0EE52D3EC20F032
:1041A000E1D7E56E1200030EEF24E8B6EF6E300E95
:0841B000EF24E8BEEF6E000CE5
:0841B8001E0EF66E000EF76EFC
:1041C000000EF86E01010900F550D76F0900F55097
:1041D000D86F03E1D76701D03DD00900F550D26F09
:1041E0000900F550D36F0900F550D46F090009009C
:1041F000F550E96E0900F550EA6E09000900090062
:10420000F550D56F0900F550D66F09000900F6CFBB
:10421000D9F1F7CFDAF1F8CFDBF1D2C1F6FFD3C194
:10422000F7FFD4C1F8FF0101D55302E1D65307E0EF
:104230000900F550EE6ED507F8E2D607F9D7D9C1D7
:10424000F6FFDAC1F7FFDBC1F8FF0101D707000E67
:06425000D85BBFD712008D
:0A4256001E502302F3CF1AF0F4CF3C
:104260001BF02402F3501B26000EF4201C6E1E507F
:104270002502F3501C26000EF4201D6E1E5026024F
:10428000F3501D261F502302F3501B26F4501C220E
:10429000000E1D221F502402F3501C26F4501D2234
:1042A0001F502502F3501D2620502302F3501C26D8
:1042B000F4501D2220502402F3501D2621502302C9
:0642C000F3501D26120060
:0A42C600FB0EE3CFF6FFFC0EE3CF82
:1042D000F7FFFD0EE3CFF8FFFE0EE3CFE9FFFF0E81
:1042E000E3CFEAFFE9CFF3FFEACFF4FF0900F5CF10
:1042F000EFFFEE66FBD71200FE0EE3CFE9FFFF0EE5
:10430000E3CFEAFFF36AF46AEE5203E0F34AF42AD9
:04431000FBD71200C5
:0C431400D9CFE6FFDACFE6FFE1CFD9FFFA
:10432000E2CFDAFFF292FD0EDBA202D0F18C01D0D7
:10433000F19CDBA002D0F18E01D0F19E9380DBAC2A
:1043400002D0F18001D0F190DBAE02D0F28801D032
:0E435000F298E552E5CFDAFFE7CFD9FF120071
:02435E00D9CFB5
:10436000E6FFDACFE6FFE1CFD9FFE2CFDAFFFD0EBD
:10437000DB507E0BCD6EFD0EDBAC02D0CD8E01D0BE
:10438000CD9ECF6ACE6A9E90DBAE02D09D8001D0DA
:104390009D90CD80E552E5CFDAFFE7CFD9FF12003F
:1043A000D9CFE6FFDACFE6FFE1CFD9FFE2CFDAFFE0
:1043B000E652E652FC0EDBCFDEFFDBCFDDFF010E67
:1043C000DB50CF6EDF50CE6EE552E552E552E5CFC1
:0843D000DAFFE7CFD9FF12006C
:0843D800FF0EE350336EEF0EFF
:1043E00001D0F30EE76EE72EF3EF21F00C0E326EE4
:1043F000E76AE72EF9EF21F0322EF8EF21F0332EA5
:06440000F1EF21F01200B3
:0A4406001D6A1C6A100EE76ED890C4
:10441000203621361C361D3625501C5C26501D5872
:1044200005E325501C5E26501D5A202AE72EF0D7A2
:02443000120078
:0E443200000EF36E00EE00F0060E01D8120030
:10444000EA6002D0EE6AFCD7F350E9601200EE6A2F
:02445000FCD797
:0E44520015EE00F025EE00F0F86A199CDCEC87
:0E44600020F003EC00F09AEC11F0FBD71200F4
:02446E00F36AEF
:10447000F46AF32A0F0B05E0D890F336F436E8041B
:04448000FBE112004A
:0C448400313233343536373839303132BC
:10449000333435360000000000000000000000004A
:1044A000000000000000000000000000000000000C
:1044B0000000003132333435363738393031323359
:1044C0003435363738393031323334353637383998
:1044D00030313233343536373839303132333435A0
:1044E000004D0150524F4A455420433138203A562E
:1044F000656C6F5F3138463235382E6D63700D0054
:1045000000000000000000000000000000000000AB
:10451000000000000000000000000000000000009B
:104520000000005F0100523D6A3D8C3D9E3DB43D60
:10453000CA3DD83DEB3D083E193E293E393E493E35
:10454000593E693E793E893E993EA93EB93EC93EF3
:06455000D93EE93EF93EF0
:020000040030CA
:01000100FA04
:01000200F409
:01000300FEFE
:01000600FBFE
:0200000400F00A
:1000000030202020202020202020202020202020E0
:100010002020202020202020202020202020200000
:1000200030202020202020202020202020202020C0
:1000300020202020202020202020202020202000E0
:1000400030202020202020202020202020202020A0
:1000500020202020202020202020202020202000C0
:100060003020202020202020202020202020202080
:1000700020202020202020202020202020202000A0
:100080003020202020202020202020202020202060
:100090002020202020202020202020202020200080
:1000A0003020202020202020202020202020202040
:1000B0002020202020202020202020202020200060
:1000C0003020202020202020202020202020202020
:1000D0002020202020202020202020202020200040
:1000E0003020202020202020202020202020202000
:1000F0002020202020202020202020202020200020
:00000001FF
